:100000000C9438000C9453000C9453000C9453003F
:100010000C947E040C9453000C9453000C945300E5
:100020000C9453000C94E3030C9453000C94530071
:100030000C9453000C9453000C9453000C945300F4
:100040000C940F040C9453000C9453000C943F0731
:100050000C94400E0C9453000C9453000C945300D9
:100060000C9453000C9453000C9453000C945300C4
:1000700011241FBECFEFD4E0DEBFCDBF12E0A0E061
:10008000B1E0E8E1F9E302C005900D92A038B107B4
:10009000D9F714E0A0E8B2E001C01D92A230B10788
:1000A000E1F70C940F060C9400009091AC02292FFC
:1000B000221F2227221F892F82958695869583707D
:1000C0002827892F82958F702827892F86958695D6
:1000D00028272170892F9927880F991F282B209373
:1000E000AC02822F99270895FF920F931F93F894E3
:1000F000809182028150823000F180918D028630A1
:1001000010F010928D0280918D0280FF02C09498B1
:1001100004C0949A88EF0E94230880918D0288235E
:1001200039F080918D028F5F80938D02789447C360
:1001300080918D028F5F80938D028091810280FF7C
:10014000E4C18091D70299278830910541F1893027
:10015000910594F48330910509F48AC084309105A7
:100160001CF4019721F10AC38530910509F41EC1E1
:10017000079709F4A1C002C38B30910509F49CC014
:100180008C30910524F4099709F410C1F7C28D3021
:10019000910509F40BC10F9709F48EC0EFC280E0FE
:1001A0000E947E0F8091A7020E94EB08E7C2809117
:1001B0008D03882321F480918203882361F090913C
:1001C000A7029F3F41F0991F9927991F8091A30291
:1001D000892B0E947E0F80918203882309F4CEC26E
:1001E00080918A03803150F480918A03E82FFF27A1
:1001F000E057FC4F80818F3F09F0C0C210928A0304
:10020000809189038F5F8093890380918903803176
:1002100068F480918903E82FFF27EE0FFF1FEE5946
:10022000FC4F808191818F5F9F4F11F41092890361
:1002300080918903E82FFF27EE0FFF1FEE59FC4F37
:1002400080819181909385038093840380918403BE
:10025000909185038F5F9F4F21F48FEF80939003E0
:100260008DC20E940A1180939D020E94EE0B86C2ED
:1002700080918D03882309F481C28091A7028F3F6A
:1002800029F0881F8827881F0E947E0F80918A038B
:100290008F5F80938A0380918A03803150F480912C
:1002A0008A03E82FFF27E057FC4F80818F3F09F03A
:1002B00065C210928A0362C28091E103882309F427
:1002C0005DC29091A7029F3F41F0991F9927991F06
:1002D0008091A302892B0E947E0F2091A702822F7A
:1002E00099278F739070892B21F080919D02820F46
:1002F00001C0822F0E94EB0880918A03803150F464
:1003000080918A03E82FFF27E057FC4F80818F3FC1
:1003100009F034C210928A038091E0038F5F8093CA
:10032000E0038091E003803248F48091E003E82FFD
:10033000FF27E054FC4F80818F3F11F41092E003BF
:1003400060EC73E080EA93E00E94D718882331F0D4
:100350009091A1028091A0029817A1F0A0EAB3E0C9
:10036000E0ECF3E09FE18D918193915097FFFBCFFB
:100370001092E00310929D0210929C020E94170DB1
:100380000E94C00D8091A0028093A10280919C02E6
:1003900080939D028091E003E82FFF27E054FC4FFB
:1003A00060818091A1020E945115E8C18091E10312
:1003B000882309F4E3C19091A7029F3F41F0991F60
:1003C0009927991F8091A302892B0E947E0F20916B
:1003D000A702822F99278F739070892B59F0109163
:1003E0009D02120F80918403909185030E94F51065
:1003F000810F01C0822F0E94EB0880918A03803117
:1004000050F480918A03E82FFF27E057FC4F80814A
:100410008F3F09F0B3C110928A0380918903803124
:1004200070F480918903E82FFF27EE0FFF1FEE592C
:10043000FC4F808191818F5F9F4F09F050C01092D7
:1004400089038091E0038F5F8093E0038091E00354
:10045000803248F48091E003E82FFF27E054FC4FFE
:1004600080818F3F59F51092E00360EC73E080EAE1
:1004700093E00E94D718882331F09091A1028091D7
:10048000A002981791F0A0EAB3E0E0ECF3E09FE15E
:100490008D918193915097FFFBCF10929D02109206
:1004A0009C020E94170D0E94C00D8091A0028093B3
:1004B000A10280919C0280939D0205C08091E0037F
:1004C0008F5F8093E0038091E003E82FFF27E054E3
:1004D000FC4F60818091A1020E94961105C080911D
:1004E00089038F5F8093890380918903E82FFF2719
:1004F000EE0FFF1FEE59FC4F808191819093850391
:10050000809384030E940A1139C18091D7029927F0
:100510008830910541F18930910594F4833091053B
:1005200009F48EC0843091051CF4019771F126C145
:100530008530910509F4BFC0079709F4B2C01EC108
:100540008B30910509F4ADC08C30910524F40997E6
:1005500009F4B1C013C18D30910509F4ACC00F97F7
:1005600009F49FC00BC18091A70280938002809103
:10057000A6028093A7020E9455008093A602809154
:10058000A70240E0642F8F73F3C080918D0388230E
:1005900029F480918203882309F4F0C080918D03AF
:1005A000882379F080918A03803148F480918A030E
:1005B000E82FFF27E057FC4F80818F3F11F4109206
:1005C0008A036091A7026093800280918A03E82FDA
:1005D000FF27E057FC4F8F5F80938A03E081E09311
:1005E000A702EF3F09F4CAC08091A202882319F044
:1005F000E07CE093A7022091A702822F99278F73B6
:100600009070422F4295469546954370661F662727
:10061000661F2F73892B59F041708091A402482BDB
:100620008091A302682B80919D02820F37C0417098
:100630008091A402482B8091A302682B822F2EC0A8
:1006400080918D03882309F499C00E94EE0B80915C
:100650008A030E94120C8091A702809380028091ED
:100660008A03E82FFF27E057FC4F80818093A70281
:100670008F3F09F483C00E94570D2091A702922F4B
:100680009295969596959370917080918002881FAF
:100690008827881F492F682F822F8F730E94630F2E
:1006A0006DC08091E103882331F00E94EE0B8091B0
:1006B0008A030E94120C8091E103882309F45EC032
:1006C0000091A7020093800280918A03E82FFF2700
:1006D000E057FC4F8F5F80938A03E081E093A7028D
:1006E000EF3F09F44BC08091A202882319F0E07C0F
:1006F000E093A7022091A702822F99278F73907011
:10070000422F4295469546954370602F661F662797
:10071000661F2F73892B21F151E0F52EF422809171
:10072000A402F82A0091A302062B10919D02120F39
:1007300080918403909185030E94F5104F2D602FC6
:10074000810F0E94630F1091A70280919D02180FE4
:1007500080918403909185030E94F510810F0CC055
:1007600041708091A402482B8091A302682B822FB4
:100770000E94630F8091A7020E94C70880918102A6
:10078000843030F485E20E944B0B0E94B20D09C008
:1007900080918102883028F485E20E94AD0B0E948E
:1007A000A50D0E94940D809181028F5F809381023C
:1007B00080918102883010F01092810278941F910C
:1007C0000F91FF9008951F920F920FB60F92112470
:1007D0002F933F934F935F936F937F938F939F9349
:1007E000AF93BF93EF93FF938091AD029091AE02D0
:1007F00090938900809388000E947400FF91EF918C
:10080000BF91AF919F918F917F916F915F914F9128
:100810003F912F910F900FBE0F901F9018951F9230
:100820000F920FB60F9211242F933F934F935F9324
:100830006F937F938F939F93AF93BF93CF93EF93D8
:10084000FF9380918E028F3F29F080918E028F5FFF
:1008500080938E0280919E0290919F028F5F9F4FA6
:1008600049F080919E0290919F02019690939F0281
:1008700080939E0280918B0290918C02892B81F053
:1008800080918B0290918C02019790938C028093BF
:100890008B0280918B0290918C02892B09F49498A1
:1008A000809182028130C1F4C0B3C295CF70C17013
:1008B00080918802882371F4CC2361F080918C02AE
:1008C00090918D02019690938D0280938C0288EF17
:1008D0000E942308C0938802FF91EF91CF91BF91AE
:1008E000AF919F918F917F916F915F914F913F91C8
:1008F0002F910F900FBE0F901F9018951F920F927F
:100900000FB60F9211242F933F938F939F9329B388
:1009100023708091AF02281791F1833041F4223087
:1009200099F48091AA029091AB02019709C082309C
:1009300059F4233049F48091AA029091AB020196B8
:100940009093AB028093AA028091AA029091AB028D
:100950008D52914030F08CE291E09093AB02809305
:10096000AA028091AA029091AB02449730F484E1EC
:1009700090E09093AB028093AA022093AF029F91E4
:100980008F913F912F910F900FBE0F901F90189550
:1009900043E350E081B1886981B940B920E030E09B
:1009A0002CBF4FE150E08AB188698AB949B920BDAE
:1009B00080EC8ABB8CE38BBB8BEB87BB18BA8FEFC9
:1009C00084BB81BB86B981E58DB9089589B7816003
:1009D00089BF8BE083BF8AEF81BF089580917D003E
:1009E000846080937D00089585E20E94AD0B809124
:1009F0007D008B7F80937D000895E199FECF9FBBA2
:100A00008EBBE09A8DB39927089580917D008695DD
:100A100086959927817090700895E199FECF9FBBCC
:100A20008EBB6DBBF894E29AE19A789408950F9387
:100A30001F93CF93DF938C0181E00D32180710F0E4
:100A40000CE211E00431110510F404E110E0109300
:100A5000A9020093A8021093AB020093AA02812F6F
:100A60009927682F85E090E00E940D056091A8020B
:100A700086E090E00E940D058091A8029091A90265
:100A80000E94010EC0E0D0E7E8E3F9E398014427B3
:100A90005527BE01CF010E946A1CFA01E90193E0CB
:100AA000F695E795D795C7959A95D1F7BE01CF01F1
:100AB00026E030E040E050E00E946A1CFA01E901C3
:100AC000CA01AA27BB279C01009731F4D093AE023C
:100AD000C093AD0281E061C0887F892B69F403E097
:100AE000F695E795D795C7950A95D1F7D093AE02BD
:100AF000C093AD0282E051C0C901807F892B69F4A7
:100B000014E0F695E795D795C7951A95D1F7D09348
:100B1000AE02C093AD0286E040C0C901807E892B41
:100B200069F4B5E0F695E795D795C795BA95D1F7ED
:100B3000D093AE02C093AD0287E02FC0C901807C84
:100B4000892B69F4A6E0F695E795D795C795AA9500
:100B5000D1F7D093AE02C093AD0283E01EC0C901AD
:100B60008070892B51F48D2F9E2FAF2FBB27909330
:100B7000AE028093AD0284E010C020703C7F232B36
:100B800079F46AE0F695E795D795C7956A95D1F718
:100B9000D093AE02C093AD0285E080938A0002C07C
:100BA00010928A008091AD029091AE02909581954D
:100BB0009F4F9093AE028093AD02909389008093F3
:100BC0008800DF91CF911F910F9108950F931F938C
:100BD00080916B00816080936B0080916B008260DC
:100BE00080936B008BB788608BBF85E090E00E949C
:100BF000FD049927182F002786E090E00E94FD044D
:100C00009927802B912B0E941705109281028091C9
:100C10007D00846080937D001F910F910895CFEF38
:100C2000D4E0DEBFCDBF0E94C8040E94E6050E944A
:100C3000E6048091A8028093AC020E9465090E949C
:100C4000910778940E94B1098091D7029927883042
:100C5000910509F453C089309105CCF48330910596
:100C600071F18430910554F48130910569F182303D
:100C700091050CF052C0892BB9F1E4CF8530910574
:100C800059F185309105ACF1079731F1DBCF8C300C
:100C9000910509F442C08D3091051CF40A97E9F1E1
:100CA0001DC08E30910531F08E30910594F00F9774
:100CB00081F0C8CF109282020E94580FC3CF1092C9
:100CC00082020E940616BECF109282020E94031278
:100CD000B9CF1092820205C081E001C082E080930A
:100CE00082020E94F018AECF109282020E94350854
:100CF000A9CF109282020E94850FA4CF1092820287
:100D00000E94EE040E94D90B0E94B1098091D70283
:100D10008830D1F30E94F40495CF0E94D90B0E9431
:100D2000940D90CF159BFECF83B980E090E008959D
:100D3000CF93DF93EC018881882331F089910E9461
:100D4000920688818823D1F7DF91CF9108950F9380
:100D50001F93CF93DF93EC0100E117E2CE01B801BE
:100D60000E94561C6115710581F0862F805D0E94DE
:100D70009206CE01B8010E94561CEC01C8016AE03F
:100D800070E00E94561C8B010EC0CE01B8010E947B
:100D9000561CEC01C8016AE070E00E94561C8B01F1
:100DA0006A307105D8F601151105A9F0CE01B80118
:100DB0000E94561CCB01805D0E949206CE01B801B4
:100DC0000E94561CEC01C8016AE070E00E94561CAB
:100DD0008B01672B59F7DF91CF911F910F910895E8
:100DE0008F708A3010F4805D01C0895C0E94920689
:100DF00008950895CF93DF93EC01892F9927829569
:100E00008F70009711F00E94F0068D2F99270097A0
:100E100011F00E94F006CE0144E0969587954A9520
:100E2000E1F7009711F00E94F0068C2F0E94F00667
:100E3000DF91CF91089582B1992787FD90958827FA
:100E4000990F881F99270895179BFECF83B1992783
:100E5000089520EA3FE0E22FF32F3197F1F78A95CA
:100E6000D1F708958AEF0E9429078AEF0E94290787
:100E70008AEF0E9429078AEF0E94290708951F928E
:100E80000F920FB60F9211248F939F93EF93FF93BE
:100E90009CB1983FB1F480918202813021F0949A04
:100EA00085E080938B028091E103882349F1809152
:100EB000830290918402019690938402809383022E
:100EC0001FC080918602E82FFF27EF54FD4F9083CB
:100ED0008F5F80938602809186028F718093860255
:100EE0009091860280918702981751F48091870231
:100EF0008F5F80938702809187028F718093870232
:100F0000FF91EF919F918F910F900FBE0F901F90C7
:100F1000189599270E94FD04803108F08FE09927E9
:100F2000089583E00E9489078093D10284E00E94A3
:100F300089078093B002089590918702809186027C
:100F4000981719F081E090E0089580E090E008950E
:100F5000089590918702809186029817D1F3F894B2
:100F600080918702E82FFF27EF54FD4F8F5F80931A
:100F700087029081809187028F7180938702789495
:100F8000892F992708950E949C07892BC1F00E9400
:100F9000A90787FF14C0682F62956F70482F5527E7
:100FA0006F3059F09A012F7030708091D1029927DB
:100FB0002817390721F460938502CA01089580E05B
:100FC00090E00895089590918002891741F480E09F
:100FD0000E947E0F0E94290D8FEF8093800208955A
:100FE0000895FF920F931F93CF93C82F00E0F02E28
:100FF000662321F4602F0E94E30720C080918002C5
:101000008F3F09F001E0653610F081E0F82E1C2FCB
:1010100019514F2D602F812F0E94630F812F0E9445
:10102000570D81E0F81619F48F2D0E944B0B0130FB
:1010300019F482E00E944B0BC0938002CF911F9164
:101040000F91FF9008955D9BFECF8CB980E090E0FA
:1010500008958091B002806B0E9423088BE70E9464
:10106000230880E00E94230808950F931F93CF93D5
:101070000E94F4040E94EE0B8091D1020E94120C97
:10108000C091DE028FEF809380020E94B1098091AF
:10109000D702882319F00E94290875C00E94450BC9
:1010A000882339F14C2F55278091DE02992701962C
:1010B0009C01207F3170821B930B2091D102481735
:1010C000590721F4222339F0215003C02F3019F0A1
:1010D0002F5F2093D1026091D10283E090E00E94C3
:1010E0000D050E94EE0B8091D1020E94120CC0915E
:1010F000DE020E949C07892B41F20E94A907082F5B
:1011000087FFC3CF482F42954F704F3051F099273A
:101110008F7090702091D10233278217930709F0C6
:10112000B4CF40938502842F99278930910551F0DF
:101130008A3091051CF4089779F018C00E9709F4CD
:10114000A4CF14C00E94A9078C010E94A907682F90
:10115000802F0E94F10799CF0E94A9078C010E945D
:10116000A907682F802F0E94E3078FCF83E091E0CB
:101170000E949806802F99270E94FA068DE191E03F
:101180000E94980682CFCF911F910F910895CF931F
:10119000C82F8091B00280690E9423088C2F992764
:1011A0008F739070892B11F480E003C08C2F8F73A4
:1011B000875E0E9423088C2F829586958695837082
:1011C00080FF03C08091020102C0809100010E9453
:1011D0002308CF910895CF93C82F8091B0028068E3
:1011E0000E9423088C2F99278F739070892B11F4FC
:1011F00080E003C0CF738C2F875E0E94230880910C
:1012000001010E942308CF910895809182028230CB
:1012100029F08CEF0E9423080E9429080895089560
:10122000CF930E940505C82F809182028130D1F0B2
:10123000CC2311F00E94F4049498979A85E00E94C0
:1012400029078091AD029091AE020A979093890090
:101250008093880010928D0210928102CC2311F0AD
:101260000E94EE04CF91089580918202813009F0AE
:1012700097980895089590B3991F9927991F809181
:101280008A02882339F4992329F090938A0281E015
:1012900090E0089590938A0280E090E00895089588
:1012A00090B3991F9927991F80918902882339F05B
:1012B000992329F49093890281E090E00895909316
:1012C000890280E090E00895089581B3806F81BB2A
:1012D00082B38F7082BB08958FE091B3982391BB46
:1012E00092B3982392BB0895DE980895AC01F894C8
:1012F000C0980000000000000000C09A20E01FB865
:10130000779BFECFFA01E20FF11D8FB180832F5F33
:101310002330A8F37894089599B3969596959F7085
:10132000292F269526952695892F86958270282B1C
:10133000892F9927880F991F382F3470232B880FF6
:10134000991F880F991F8870282B8FE0821B99277F
:101350000895DE9A089589B3869586958F709927AA
:101360000895AF92BF92CF92DF92EF92FF920F93C8
:101370001F93CF93DF93CDB7DEB726970FB6F894C0
:10138000DEBF0FBECDBF2091AA023091AB0280918B
:10139000A8029091A9022817390731F08091AA027A
:1013A0009091AB020E941705ABEDB2E0E4EDF2E0E4
:1013B00042E011921D92415047FFFBCF80918E0277
:1013C000843108F490C010928E020E947409CE01FC
:1013D00001960E9476098091D8028C838091D9026F
:1013E0008D838091DA028E8340E001E010E05E019F
:1013F000A00EB11E842F869586958695A82FBB27B3
:10140000BD0168527D4F842F8770980102C0220F62
:10141000331F8A95E2F7C901FB013081232F28236E
:10142000FD01E152FD4FE081E823AA0DBB1DAC9107
:10143000A8234F5F8095222319F03823EA2B02C09E
:101440003823EA233E2BFB013083483198F20E9477
:101450008C09482F8091DE02481749F08091D30211
:10146000481729F44093DE0281E080938F02409375
:10147000D3020E94A9096BEDC62E62E0D62E54ED70
:10148000E52E52E0F52E08ED12E0BE016C5F7F4FB5
:10149000AFEDB2E042E0F50181915F018D93FB0178
:1014A0002191BF01F80181918F01922F9827892303
:1014B000F70181937F019223F60191936F014150CF
:1014C00047FFE9CF0E94AB09482F8091D702481708
:1014D00031F08091D202481711F44093D702409323
:1014E000D2020E94940D26960FB6F894DEBF0FBE6E
:1014F000CDBFDF91CF911F910F91FF90EF90DF90C3
:10150000CF90BF90AF900895282F883118F080E0D9
:1015100090E00895869586958695E82FFF27E852F6
:10152000FD4F80819927277002C0959587952A9550
:10153000E2F79C012170307080FF03C081E090E0F1
:101540000895C90108950895282F883118F080E082
:1015500090E00895869586958695E82FFF27EC52B2
:10156000FD4F80819927277002C0959587952A9510
:10157000E2F79C012170307080FF03C081E090E0B1
:101580000895C90108950895282F883118F080E042
:1015900090E00895869586958695E82FFF27E55279
:1015A000FD4F80819927277002C0959587952A95D0
:1015B000E2F79C012170307080FF03C081E090E071
:1015C0000895C901089508958091D802882359F497
:1015D0008091D902882339F48091DA02882319F4A2
:1015E00081E090E0089580E090E008950895FF92F2
:1015F0000F931F93CF93DF93FF2400E010E0C8E226
:10160000D1E088810E94840A882311F0C80109C0B2
:10161000F39421960F5F1F4F8CE08F1594F78FEF97
:101620009FEFDF91CF911F910F91FF900895CF937E
:10163000C0E0EC2FFF27E05EFE4F80810E94840A0D
:10164000EC2FEF5F882319F08E2F992705C0CE2F3E
:10165000E83078F380E090E0CF910895CF93C0E038
:10166000EC2FFF27E05EFE4F80810E94A40AEC2F42
:10167000EF5F882319F08E2F992705C0CE2FE83011
:1016800078F380E090E0CF91089580918F021092DE
:101690008F0299270895282F883290F48695869591
:1016A0008695E82FFF27EB56FD4F277081E090E0ED
:1016B00002C0880F991F2A95E2F72081282B2083EA
:1016C00008950895282F883290F4869586958695FA
:1016D000E82FFF27E057FD4F277081E090E002C020
:1016E000880F991F2A95E2F72081282B20830895DF
:1016F0000895282F8832A0F4869586958695E82F40
:10170000FF27E057FD4F277081E090E002C0880F6F
:10171000991F2A95E2F7982F9095808189238083DD
:1017200008950895282F883218F080E090E00895F9
:10173000869586958695E82FFF27E057FD4F277001
:1017400081E090E002C0880F991F2A95E2F720817E
:101750002823822F992708950895282F8832A0F4EE
:10176000869586958695E82FFF27EB56FD4F2770C7
:1017700081E090E002C0880F991F2A95E2F7982F28
:10178000909580818923808308950895282F8695D8
:1017900086958695E5E9F2E0E80FF11D80819927AD
:1017A000277002C0959587952A95E2F78170907011
:1017B0000895109299021092980210929702109236
:1017C0009602109295021092940210929302109237
:1017D0009202109291021092900208950F931F931B
:1017E000CF9302E611E0CFE0F80181918F010E94D2
:1017F000AD0BC150C7FFF8CFCF911F910F91089546
:101800000F931F93CF9302E611E0CFE0F80181918F
:101810008F010E94790BC150C7FFF8CFCF911F9164
:101820000F910895803138F4E82FFF27EE59FE4FCD
:1018300080810E944B0B08950895803138F4E82F81
:10184000FF27EE59FE4F80810E94620B0895089594
:10185000803118F020E030E009C0E82FFF27EE5972
:10186000FE4F80810E94C60B282F3327C90108959F
:10187000803118F080E090E00895E82FFF27EE59BE
:10188000FE4F80810E94920B992708950895883118
:1018900038F4E82FFF27E65BFE4F80810E944B0B58
:1018A00008950895883138F4E82FFF27E65BFE4F4E
:1018B00080810E94620B08950895883138F4E82FE2
:1018C000FF27E65BFE4F80810E94AD0B08950895CF
:1018D0000F931F93CF930AE411E0C7E1F8018191C0
:1018E0008F010E94AD0BC150C7FFF8CFCF911F9160
:1018F0000F910895E82F8150883030F4FF27EF5B77
:10190000FE4F80810E944B0B089508951F93CF9343
:10191000182F81E0E82FFF27C82FCF5F811731F400
:10192000EF5BFE4F80810E944B0B05C0EF5BFE4FCB
:1019300080810E94AD0B8C2FC93060F3CF911F9135
:101940000895E82F8150883030F4FF27EF5BFE4F79
:1019500080810E94AD0B08950895E82F8150883052
:1019600030F4FF27EF5BFE4F80810E94790B0895D2
:101970000895E82F8150883030F4FF27EF5BFE4F49
:1019800080810E94620B08950895E82F815088306D
:1019900040F4FF27EF5BFE4F80810E94920B992756
:1019A000089580E090E008950895E82F81508830F0
:1019B00048F4FF27EF5BFE4F80810E94C60B282F63
:1019C000332702C020E030E0C90108950F931F9330
:1019D000CF9302E411E0C7E0F80181918F010E94EA
:1019E000AD0BC150C7FFF8CFCF911F910F91089554
:1019F0008D3038F4E82FFF27EB5CFE4F80810E948A
:101A00004B0B089508958D3038F4E82FFF27EB5CD9
:101A1000FE4F80810E94620B08950895E5E3F1E096
:101A2000E80FF11D80810E94920B992708950F9372
:101A30001F93CF9305E311E0CCE0F80181918F0172
:101A40000E94AD0BC150C7FFF8CFCF911F910F91EE
:101A500008950E94170D84E00E94AD0B83E00E9460
:101A6000AD0B88E00E94AD0B81E00E94AD0B82E0DF
:101A70000E94AD0B0895CF93C82F84E00E94AD0B58
:101A8000C23021F483E00E94620B0FC083E00E9409
:101A9000AD0B83E00E94790BC13011F483E003C0E9
:101AA000CF3F19F484E00E944B0BCF910895CF9360
:101AB000C82F0E94290DC7FF03C086E10E94470C72
:101AC0008C2F829586958695837080FF03C085E173
:101AD0000E94470CCF7311F48C2F15C0C73110F43E
:101AE0008FEF11C0C43218F4CC5080E00CC0C0336A
:101AF00018F4C85181E007C0CC3318F4C45282E016
:101B000002C083E0C0530E943B0DCC2321F484E14A
:101B10000E94470C07C0EC2FFF27E65DFE4F808137
:101B20000E944B0BCF910895F894DF98E5E9F2E01D
:101B300080818FB9779BFECF319682E0E939F80733
:101B4000B9F3B4F3DF9A78940895A0E9B2E0E5E937
:101B5000F2E024E080819D91892B8193215027FF21
:101B6000F9CF0895A0E9B2E0E5E9F2E024E09D9123
:101B70009095808189238193215027FFF8CF089584
:101B8000A0E9B2E0E5E9F2E034E020819C91822F07
:101B9000892319F09095292320831D923150319685
:101BA00037FFF3CF0895AC0120E0322F61157105A6
:101BB00081F0FA01E30FF11D80812827E22FFF2732
:101BC000EE58FE4F20813F5F832F99278617970796
:101BD00080F3822F992708950F931F93CF93DF935C
:101BE0006115710549F08C01EB01F80181918F01BC
:101BF0000E9492062197C9F7DF91CF911F910F9113
:101C000008950F931F939C0102EE12E082E48093EB
:101C1000E2021092E30282E08093E402832F99278C
:101C20008093E5022093E60265E070E0C8010E941F
:101C3000D30D8093E70266E070E0C8010E94EC0DCE
:101C40001F910F9108950F931F9302EE12E090E8F9
:101C50009093E2021092E30291E09093E402809369
:101C6000E50264E070E0C8010E94D30D8093E602B3
:101C700065E070E0C8010E94EC0D1F910F9108957E
:101C80001F920F920FB60F921124EF92FF921F93A3
:101C90002F933F934F935F936F937F938F939F9374
:101CA000AF93BF93CF93DF93EF93FF9393B1809163
:101CB0007202882309F4E4C080919B02803448F4C6
:101CC000E82FFF27EE5DFC4F90838F5F80939B0290
:101CD00004C00E94230E10929B0220919B0223308D
:101CE00008F4CEC0F090220380912303682F772759
:101CF000762F6627809124039927682B792B332729
:101D0000CB0104962817390708F4BAC0FB01EE5D31
:101D1000FC4F1381EB012396BE0182E293E00E9407
:101D2000D30D181791F0BE0182E293E00E94D30D0B
:101D300099270E94FA0610929B0280E00E94230ECF
:101D40000E94EE0B0E94940D9DC08F2D992781312A
:101D5000910551F18231910544F48130910509F4E6
:101D600088C0409709F460C086C08034910521F096
:101D70008134910541F07FC08091A8029091A90221
:101D80000E94010E7BC080912403823009F073C051
:101D9000809125039927982F882720912603820F69
:101DA000911D0E9417056AC080912403823009F0BA
:101DB00062C08091250390912603C82FDD2763E040
:101DC000CC0FDD1F6A95E1F7C90FD11D89E1809322
:101DD000E2021092E30280E18093E4020F2EF5EE1E
:101DE000EF2EF2E0FF2EF02DC295D295D07FDC27AA
:101DF000C07FDC271FE0CE010E94B210F701819363
:101E00007F011150219617FFF6CF63E170E082EE5B
:101E100092E00E94D30D8093F50264E170E082EEBF
:101E200092E00E94EC0D2AC080912403823119F5C2
:101E30008091250390912603C82FDD2733E0CC0F36
:101E4000DD1F3A95E1F7C90FD11D27E2E22E23E00D
:101E5000F22E94E0CC0FDD1F9A95E1F71FE0BE0152
:101E6000F70181917F010E9473101150219617FF95
:101E7000F6CF81E001C080E00E94230E10929B0209
:101E80000E94EE0BFF91EF91DF91CF91BF91AF9147
:101E90009F918F917F916F915F914F913F912F9182
:101EA0001F91FF90EF900F900FBE0F901F9018950D
:101EB0000E94B1098091D7028E30D1F30E94D90BD4
:101EC0000E94940D089590E03A98803408F08FE3D2
:101ED000611160E4442311F440E801C0492F8823D4
:101EE00049F0862B842B85BB3A9A9F5F9832E8F3A2
:101EF000399A0895642B65BB08950895882311F0DD
:101F0000AE9A01C039983A9808957F928F929F9225
:101F1000AF92BF92CF92DF92EF92FF920F931F93F7
:101F2000CF93DF93EE24FF248824982C0E94EE04A4
:101F30000E94EE0B7090DE02670157010E94B1090A
:101F40008091D702843019F00E942908BEC0809188
:101F5000B0020E94280C882331F40E94EE0B80917D
:101F6000B0020E94120C0E94450B882309F1472DF4
:101F700055278091DE02992701969C01207F3170C0
:101F8000821B930B2091B0024817590721F422239A
:101F900039F0215003C02F3019F02F5F2093B00289
:101FA0006091B00284E090E00E940D057090DE0226
:101FB0008E2D0E943B0D992019F081E00E944B0B61
:101FC000882019F082E00E944B0B00E0C3E7D2E0CA
:101FD00088810E94A40A8823B9F0102F1A0D195E77
:101FE000492D682D812F0E94630F892D992756E076
:101FF000880F991F5A95E1F7812B0E94C708812FFE
:102000000E94570D41E0842E88810E94C40A8823D3
:1020100079F0202F2C0D295E892D992736E0880F25
:10202000991F3A95E1F7822B0E94EB080E94290D37
:102030000F5F21960D3060F28FE00E94A40A882382
:1020400051F082E0E816F104D4F40894E11CF11C8C
:102050008CE090E010C08EE00E94A40A882379F002
:102060009FEFE9169FEFF90651F04CF00894E10854
:10207000F10884EF9FEFA80EB91EC80ED91E85E1A6
:102080000E94A40A882371F080E0992009F481E07D
:10209000982E882321F081E00E944B0B03C081E041
:1020A0000E94AD0B83B399278F739070892B09F42D
:1020B00045CF0E94E40A882309F440CF80E00E94C3
:1020C0007E0F0E94290D882439CFDF91CF911F9177
:1020D0000F91FF90EF90DF90CF90BF90AF909F90C7
:1020E0008F907F900895282FF89495E0C098000075
:1020F0000000000000009FB9779BFECF00000000A9
:10210000000000001FB8779BFECF8FB1C09A00007F
:1021100000000000000080FDE9CFC0980000000032
:1021200086E08FB9779BFECF00000000C09A0000C8
:10213000000000000000C0980000000082E08FB99D
:10214000779BFECF872F99278FB9779BFECF6FB9EB
:10215000779BFECF2FB9779BFECF00000000C09A7F
:10216000789408959C01F894C0980000000083E0E2
:102170008FB9779BFECF832F99278FB9779BFECF9F
:102180002FB9779BFECF000000001FB8779BFECFD2
:102190008FB1C09A7894992708951092860310926F
:1021A0008D031092820380E00E947E0F0E94D90B63
:1021B0000E94C00D0E94450B08951092870384E28F
:1021C0000E94AD0B0E94D90B0E94C00D10928D038E
:1021D00080E00E947E0F089581E08093870384E26F
:1021E0000E944B0B0E94EE0B0895892F9927282FF0
:1021F0002F71822F992787FD909534E096958795CA
:102200003A95E1F7892B09F0206E822F992787FDF7
:102210009095089520918403277080918403909174
:102220008503F3E096958795FA95E1F7622F8F7015
:102230000E94511560918403709185039B0144278E
:102240005527DA01C90180709078A070B070892F8D
:102250009A2FAB2FBB278093A202DA01C9018070AD
:102260009074A070B070892F9A2FAB2FBB278093EA
:10227000A4022070307240705070BB27A52F942F9D
:10228000832F8093A30210928A03CB010E94F51042
:102290009927089581E08093860381E20E944B0B89
:1022A0001092A4028091A4028093A3028091A302C1
:1022B0008093A2021092820310928D038091620398
:1022C0009091630390938503809384038F5F9F4F66
:1022D00089F01092890310928A031092A7020E943B
:1022E0000A1180939D028091810280FDFCCF81E0E4
:1022F000809382030E94EE0B089580919D028823B3
:1023000021F483E00E94AD0B0CC087FF07C083E07F
:102310000E94AD0B84E00E944B0B089583E00E9465
:102320004B0B84E00E94AD0B08950895FF920F932C
:102330001F93CF93DF93C82FDD2703E0CC0FDD1F62
:102340000A95E1F7C60FD11D15E0CC0FDD1F1A95D8
:10235000E1F7BFE0FB2EC050D84F02E613E0CE01FC
:102360000E94B2109927982F8827F80180839183C3
:10237000CE0101960E94B210282F3327F8018081E8
:102380009181822B932B819391938F01FA942296C2
:10239000F7FEE5CFDF91CF911F910F91FF90089548
:1023A000FF920F931F93CF93DF93C82FDD2753E046
:1023B000CC0FDD1F5A95E1F7C60FD11D45E0CC0FBC
:1023C000DD1F4A95E1F73FE0F32E02E613E0C0502F
:1023D000D84FF80180819181892F9927BE010E94F1
:1023E00073102196F801819191918F01BE010E9495
:1023F0007310FA942196F7FEECCFDF91CF911F91E5
:102400000F91FF9008951F93CF93DF930E94EE04E6
:102410008091DE028770809383031092880310926C
:102420008703109286031092820310928D031092FC
:1024300089038FEF9FEF909385038093840310921D
:1024400082020E94EE0B0E94C00D0E94B109809191
:10245000D702813071F00E94F40410928D03109223
:10246000820380E00E947E0F0E94D90B0E94940D8F
:10247000EEC280918703882361F5809186038823CB
:1024800041F50E94450B882359F08091DE02877048
:1024900080938303609188030E9496110E94EE0B43
:1024A000809183030E94120C0E94170BC82F88236F
:1024B00059F00E94170D8C2F815080938803682F4C
:1024C000809183030E949611809188038F5F0E9400
:1024D0007A0C81E00E94A40A882379F08091860317
:1024E000882319F00E94CD1008C0809187038823AB
:1024F00011F00E94DD100E944A118091860388230A
:1025000029F480918703882309F463C080918903AB
:102510000E94380C882311F40E94C00D8091890319
:102520000E941D0C80918403909185038F5F9F4FC3
:1025300021F40E94290D80E046C080E00E94AD0B8E
:10254000809184039091850343E0969587954A9501
:10255000E1F78F700E94120C8091840390918503A3
:1025600097FF04C088E00E944B0B03C088E00E94E4
:10257000AD0B8091840390918503AA27BB273EE091
:10258000B695A795979587953A95D1F781709070F4
:10259000892B21F081E00E944B0B03C081E00E9457
:1025A000AD0B8091840390918503AA27BB272DE072
:1025B000B695A795979587952A95D1F781709070D4
:1025C000892B21F082E00E944B0B03C082E00E9425
:1025D000AD0B88E00E94A40A882331F483E00E94B6
:1025E000A40A882309F478C010918603112309F006
:1025F00073C0812F0E947E0FC0918703CC2309F402
:1026000042C088E00E94A40A8823D1F08091890307
:102610009927019640976CF480918903E82FFF2752
:10262000EE0FFF1FEE59FC4F808191818F5F9F4F0E
:1026300019F41093890330C0809189038F5F20C003
:10264000809189038823C9F4809189039927019691
:10265000409714F580918903E82FFF27EE0FFF1FA5
:10266000EE59FC4F808191818F5F9F4FA9F080913F
:1026700089038F5F80938903E7CF8091890381501D
:102680008093890309C088E00E94A40A882321F06E
:102690000E94EC10C093890380918903E82FFF27E3
:1026A000EE0FFF1FEE59FC4F8081918190938503BF
:1026B0008093840310928D038F5F9F4F69F00E9477
:1026C0000A1180939D0210928A038091810280FDFD
:1026D000FCCF81E080938D0387E10E94A40A8823C8
:1026E00039F1809187038823E9F080918903992744
:1026F0000196409764F480918903E82FFF27EE0F3D
:10270000FF1FEE59FC4F8FEF9FEF828393838FEF74
:102710009FEF90938503809384030E94DD1080E0F7
:102720000E94AD0B60918803809183030E94D011B9
:1027300080918703882309F47CC180918403909160
:1027400085038F5F9F4F09F40FC184E10E94A40AA3
:10275000882311F180918903E82FFF27EE0FFF1FD7
:10276000EE59FC4F8081918120E030E88227932749
:1027700080839183808191819093850380938403EA
:10278000AA27BB2780709078A070B070892F9A2FED
:10279000AB2FBB278093A20285E10E94A40A882365
:1027A00011F180918903E82FFF27EE0FFF1FEE59EB
:1027B000FC4F8081918120E030E482279327808341
:1027C0009183808191819093850380938403AA27CC
:1027D000BB2780709074A070B070892F9A2FAB2F98
:1027E000BB278093A40286E10E94A40A882311F1EA
:1027F00080918903E82FFF27EE0FFF1FEE59FC4F52
:102800008081918120E030E2822793278083918329
:10281000808191819093850380938403AA27BB27AD
:1028200080709072A070B070892F9A2FAB2FBB2749
:102830008093A3028FE00E94840A882331F48EE003
:102840000E94840A882309F47DC00E94F70AC82FD9
:10285000DD27C7FDD0958FE00E94A40A882329F4C4
:102860008EE00E94A40A882351F00E94C00D0E94AD
:10287000170D83E00E94AD0B84E00E94AD0B8FE04A
:102880000E94840A882349F183E00E944B0B8FEF5A
:10289000CF3FD807C9F00E94C00D2091840330912A
:1028A0008503307E9C2F8827282B392B3093850376
:1028B0002093840380918903E82FFF27EE0FFF1FE9
:1028C000EE59FC4F208331838091840390918503DE
:1028D0000E94F51080939D0232C08EE00E94840A0F
:1028E000882309F441C084E00E944B0B2FEFCF3FB7
:1028F000D207E1F00E94C00D20918403309185033E
:10290000307E2C97CF71D0709C2F8827282B392BA5
:10291000309385032093840380918903E82FFF2758
:10292000EE0FFF1FEE59FC4F20833183809184030B
:10293000909185030E94F51080939D02845F0E9410
:10294000030D12C08FE00E94C40A882329F48EE090
:102950000E94C40A882341F083E00E94AD0B84E00A
:102960000E94AD0B0E94C00D8FE00E94840A882354
:1029700009F05FC08EE00E94840A882309F059C0E4
:102980000E942E0BC82F882329F40E94450B882310
:1029900009F447C00E94E60C0E94EE0BCC2359F4C8
:1029A00080918403909185038F5F9F4F29F0C091A0
:1029B0008403C77001C0C15010928D0380E00E9453
:1029C0007E0F4091DE02242F332763E0220F331F56
:1029D0006A95E1F78C2F9927282B392B30938503A3
:1029E0002093840380918903E82FFF27EE0FFF1FB8
:1029F000EE59FC4F208331836C2F842F0E94511598
:102A000010928A031092A3028091A3028093A402E1
:102A10008091A4028093A20210929D0281E0809393
:102A20008D030E947D118091840387708F5F0E94C7
:102A3000860C80918603882309F407CD0E947D11BE
:102A40008091840387708F5F0E94860CFECCDF919B
:102A5000CF911F91089510928A0381E080938B0398
:102A600081E20E944B0B80E00E947E0F0E94EE04E8
:102A70008091810280FDFCCF81E080938D030895D9
:102A800081E08093870384E20E944B0B0E94EE0B4F
:102A900080E00E94120C0E94F40480E00E947E0FED
:102AA0000895EF92FF920F931F93CF93DF93182F08
:102AB000062F0E94940DC12FDD2723E0CC0FDD1FD0
:102AC0002A95E1F7C00FD11D94E0CC0FDD1F9A9538
:102AD000E1F780E9E82E83E0F82E1FE0CE010E94A6
:102AE000B210F70181937F011150219617FFF6CFA5
:102AF000809190038F3F41F487E1E0E9F3E01FE02C
:102B00008193115017FFFCCF0E94940DDF91CF915C
:102B10001F910F91FF90EF900895EF92FF920F9306
:102B20001F93CF93DF93182F062F0E94940DC12F70
:102B3000DD2753E0CC0FDD1F5A95E1F7C00FD11D03
:102B400040E9E42E43E0F42E34E0CC0FDD1F3A954B
:102B5000E1F71FE0BE01F70181917F010E94731030
:102B60001150219617FFF6CF0E94940DDF91CF915F
:102B70001F910F91FF90EF9008951092870384E2C8
:102B80000E94AD0B0E94680C0E94EE0B8091DE0249
:102B90000E94120C0E94EE0480E00E947E0F0895B5
:102BA0000E94F40410928D030E94680C0E94EE0BA8
:102BB0008091DE020E94120C10928B0381E20E942F
:102BC000AD0B80E00E947E0F089581E080938F031B
:102BD0000E94EE0480E00E947E0F0E94680C80E05C
:102BE0000E94620B8091DE020E94120C80918C0385
:102BF0008F5F0E947A0C089510928F0380E00E94EC
:102C0000790B0E94680C0E94EE0B0895EF92FF92E0
:102C10000F931F93CF93DF9310928C03109287032F
:102C200010928B0310928F0310928D0310928A03DF
:102C30001092A702109282020E94B1098091DE02D6
:102C400080938E0360918C030E9451150E94D90BD2
:102C50008091DE020E94120C0E94EE040E94B109D3
:102C60008091D702833081F00E94F40410928D038A
:102C700080E00E947E0F0E9434090E9405090E9494
:102C8000D90B0E94940D8CC290918E038091DE022C
:102C90009817F9F080918B03882311F00E94D015CA
:102CA00080918703882311F00E94BD159091DE0268
:102CB00090938E0380918F03882329F460918C0375
:102CC000892F0E9451150E94EE0B8091DE020E9416
:102CD000120C80918B038823F9F480918703882359
:102CE000D9F480918C038F5F0E947A0C0E94170B9D
:102CF000C82F882389F00E94170D8C2F0E947A0C10
:102D00006C2F615060938C0380918F03882321F492
:102D100080918E030E94511580E00E94A40A8823AE
:102D200099F080918B03882379F082E20E944B0B0B
:102D300000E913E0CFE00E945500F80181938F0174
:102D4000C150C7FFF8CF0CC080E00E94C40A88239E
:102D500039F080918B03882319F082E20E94AD0B39
:102D600081E00E94A40A8823A9F080918F03882320
:102D700011F00E94FC1580918B03882319F00E94AA
:102D8000D01508C080918703882311F00E94BD15DB
:102D90000E942B1580918B03882329F4809187034F
:102DA000882309F427C100918A03E02EFF24E7015C
:102DB000C057DC4F18811F7385E10E94A40A882345
:102DC00031F01F3321F0888190E48927888386E1E0
:102DD0000E94A40A882349F01F3339F0F701E05715
:102DE000FC4F808190E8892780831F3341F01123B5
:102DF00031F0173110F4CFEF0DC0143210F4C0E0F1
:102E000009C0103310F4C1E005C01C3310F4C2E057
:102E100001C0C3E084E10E94A40A811110E08FE0A8
:102E20000E94A40A882339F01F3329F0112319F0D6
:102E30001C160CF0145F8EE00E94A40A882341F057
:102E40001F3331F0112321F0CF3F11F00CF01C5053
:102E500084E00E94A40A882331F08CE0C802C001FB
:102E60001124182F195E89E00E94A40A882331F0EA
:102E70008CE0C802C0011124182F185E85E00E9462
:102E8000A40A882331F08CE0C802C0011124182F55
:102E9000175E8AE00E94A40A882331F08CE0C80201
:102EA000C0011124182F165EC3300CF063C086E0F9
:102EB0000E94A40A882331F08CE0C802C0011124CA
:102EC000182F155E87E00E94A40A882331F08CE059
:102ED000C802C0011124182F145E8BE00E94A40ABE
:102EE000882331F08CE0C802C0011124182F135E32
:102EF00081E10E94A40A882331F08CE0C802C0015D
:102F00001124182F125E8CE00E94A40A882331F04D
:102F10008CE0C802C0011124182F115E82E10E94CA
:102F2000A40A882331F08CE0C802C0011124182FB4
:102F3000105E8DE00E94A40A882331F08CE0C80264
:102F4000C0011124182F1F5D80E10E94A40A88236C
:102F500031F08CE0C802C0011124182F1E5D83E1FE
:102F60000E94A40A882331F08CE0C802C001112419
:102F7000182F1D5D202F3327F901E057FC4F80816A
:102F80008F3F11F41F3319F48081807C182BE901E5
:102F9000C057DC4F88811817F9F080918703882388
:102FA00031F080E00E947E0F81E00E9429071883A3
:102FB00080918703882381F0812F8295869586955D
:102FC00083708170912F991F9927991F482F692F1E
:102FD000812F8F730E94630F1F3F39F0812F0E9452
:102FE000570D80E00E94AD0B05C00E94290D80E0C6
:102FF0000E944B0B88E00E94A40A882331F483E0EE
:103000000E94A40A882309F49BC080918703882327
:1030100009F46AC080E00E947E0F81E00E942907C7
:1030200088E00E94A40A8823B1F080918A0399273E
:10303000019640974CF480918A03E82FFF27E057D0
:10304000FC4F80818F3F19F410928A0320C0809139
:103050008A038F5F1AC080918A03882399F4809134
:103060008A038F30A0F480918A03E82FFF27E0576E
:10307000FC4F80818F3F59F080918A038F5F80934E
:103080008A03EDCF80918A03815080938A030E9446
:10309000EE0B80918A030E94120C80918A03E82F24
:1030A000FF27E057FC4F80818093A7028F3F51F4A8
:1030B00081E00E94AD0B82E00E94AD0B80E00E9497
:1030C0004B0B3EC080E00E94AD0B8091A702982F71
:1030D00092959695969593709170282F221F22278E
:1030E000221F492F622F25C088E00E94A40A88234E
:1030F00039F1C0918B03CC2319F50E944015C09380
:103100008A0380918A03E82FFF27E057FC4FE08174
:10311000E093A702EF3FA1F08E2F829586958695CA
:10312000837081709E2F991F9927991F482F692FAF
:103130008E2F8F730E94630F8091A7020E94570DFC
:1031400087E10E94A40A882309F488CD809187032F
:10315000882381F080918A0399270196409744F44F
:1031600080918A03E82FFF27E057FC4F8FEF818380
:103170000E94BD1580918B03882311F00E94D01509
:1031800080918F03882349F060918C038091DE0247
:103190000E948D150E94FC1561CD0E94E5155ECD43
:1031A000DF91CF911F910F91FF90EF90089540E034
:1031B000DB01FC0190818C91981719F080E090E080
:1031C000089580818F3F19F481E090E008954F5F6A
:1031D00031961196403270F381E090E008950895A1
:1031E000EF92FF920F931F93CF93FF24E090D702AB
:1031F00080918202882319F40E94EE040BC00E9481
:10320000F40480918202813019F40E946C0902C09A
:103210000E9465090E94D90B0E94C00D1092C00344
:103220008091C0038093A0038FEF8093C1038091AE
:10323000C1038093A10381E00E947A0C1092E10304
:103240001092890310928A031092850310928403CE
:103250001092E00310929C0210929D020E94EE0BCD
:103260008091D7028F3021F08B3011F08730D1F46C
:103270008091DE021AC01092E1030E9434090E947C
:10328000050910929C0210929D021092A3021092C6
:10329000A2021092A4020E94D90B0E94C00D0E94AB
:1032A000940DFEC28091DE0287708093A10280930C
:1032B000A0028091DE020E94120C0E94B10980914E
:1032C000D7028E15C1F687E10E94A40A882329F14E
:1032D00080919E0290919F0286509D40D0F48091F3
:1032E0009E0290919F028E54914098F020919E02F0
:1032F00030919F0280E69AEEB9010E94561C7093AD
:103300009F0260939E0280919E0290919F020E9474
:10331000170510929F0210929E0280E00E94A40A5C
:10332000882349F00E94170D0E94C00D82E20E947E
:103330004B0B1092A50280E00E94C40A882329F159
:10334000A2EEB3E0E0EAF3E0CFE18D918193C150CA
:10335000C7FFFBCF8091E1038823A1F4A0EAB3E08B
:10336000E0ECF3E0CFE18D918193C150C7FFFBCF3B
:1033700080919C0280939D0283E00E94AD0B84E0CB
:103380000E94AD0B82E20E94AD0B80E00E94840A95
:10339000882361F1C0E08091A502C81760F4EC2F8A
:1033A000FF27EE51FC4F8081883028F48F5F0E9408
:1033B0007A0CCF5FF0CF0E942E0BC82F882309F420
:1033C0004EC18091A502803208F049C1E82FFF2745
:1033D000EE51FC4FC150C0838F5F8093A502E82F50
:1033E000FF27EE51FC4F8FEF808339C18FE00E94A1
:1033F000840A882331F48EE00E94840A882309F429
:103400006DC00E94F70AC82F8FE00E94A40A88238B
:1034100029F48EE00E94A40A882339F00E94170D37
:103420000E94C00D82E20E94AD0B8FE00E94840AD0
:10343000882301F184E00E94AD0B83E00E944B0BD6
:10344000CF3F11F0C0939C0280919D0287FD0AC07E
:103450000E940E0D882331F40E94C00D80919D02C0
:103460000E94030D90919C0280919D02981761F13A
:10347000892F28C08EE00E94840A882329F183E0E6
:103480000E94AD0B84E00E944B0BCF3F19F0CC5053
:10349000C0939C0280919D02181664F0845F0E9484
:1034A0000E0D882339F40E94C00D80919D02845F27
:1034B0000E94030D90919C0280919D02981721F02B
:1034C000892F845F0E94F80C8091E103882309F022
:1034D000C6C080919C0280939D02C1C08FE00E9473
:1034E000C40A882329F48EE00E94C40A882321F0AC
:1034F0000E94170D0E94C00D0E94170BC82F882331
:1035000031F40E94450B882309F446C01FC00E9475
:10351000E60CC150C093A0038091A0038093E20306
:103520008FEF8093A1038091A1038093E3038091A7
:10353000E103882319F5A0EAB3E0E0ECF3E0CFE182
:103540008D918193C150C7FFFBCF18C08091D702E6
:103550008F3021F08B3011F0873019F48091DE022A
:1035600003C08091DE0287708093A0028091E10306
:10357000882321F48091A0028093A1028091E1032D
:10358000882351F40E94EE0B8091A0020E94120C3D
:1035900080919C0280939D0260EC73E080EA93E04E
:1035A0000E94D7188823F9F48091A1038F3F49F432
:1035B0008091C1038F3F29F48091C0038F5F0E94E7
:1035C000B90CC0E000EA13E0F8018081893008F00E
:1035D00044C0D8018D918D018F5F0E947A0CCF5F1E
:1035E000C03290F33AC0C0E000EC13E0F8018081F3
:1035F000893098F58091E1038823E1F08091E00320
:10360000E82FFF27E054FC4FD8019C918081981748
:1036100089F48C918F5F0E94C50C8823C9F4F8014E
:1036200080818F5F0E94A10CD8018C918F5F0E94D6
:10363000B90C0EC0F80180818F5F0E94C50C8823F1
:1036400011F00E94C00DD8018C918F5F0E947A0CFE
:10365000CF5F0F5F1F4FC03248F20E947D118091F3
:10366000E103882351F180918202823089F48091B4
:1036700083029091840218161906FCF4809183024B
:10368000909184020397909384028093830212C0E6
:10369000813099F480918C0290918D021816190650
:1036A00064F480918C0290918D02039790938D0227
:1036B00080938C020E94740000CE8091820282303E
:1036C00019F40E94C307F82E80918202882349F4DE
:1036D00081E00E94A40A882321F08091E1038823DD
:1036E00071F480918202823021F4BCEFFB1639F034
:1036F0002BC0813049F50E945009882329F110928E
:10370000E10380E00E947E0F0E9405098091820201
:10371000813011F00E94340981E20E94AD0B0E94B9
:10372000C00D0E94EE0B8091D7028F3021F08B30BC
:1037300011F0873019F48091DE0203C08091DE021F
:1037400087700E94120C68C080918202882349F41D
:1037500081E00E94A40A882321F08091E10388235C
:1037600089F080918202823029F48F2D8A5F823025
:1037700048F052C0813009F04FC00E943B098823B5
:1037800009F44AC081E20E944B0B8091D7028F302E
:1037900021F08B3011F0873039F46091C0038091B3
:1037A000DE020E94511511C08091DE026091C003BB
:1037B00087700E94961180916203909163039093A9
:1037C0008503809384030E940A111092A7028091BE
:1037D0008202823019F4EBEFFE1631F01092E00312
:1037E00010928A031092890310928102109284022F
:1037F0001092830210928D0210928D0210928C0210
:1038000081E08093E1038AEF0E9423088091820285
:10381000813011F00E94100986E10E94A40A8823D9
:1038200089F090E08091A302882309F491E09093BD
:10383000A302992321F082E00E944B0B03C082E097
:103840000E94AD0B85E10E94A40A882389F090E0D4
:103850008091A402882309F491E09093A402992313
:1038600021F081E00E944B0B03C081E00E94AD0B70
:1038700084E10E94A40A882309F41FCD90E080917E
:10388000A202882309F491E09093A202992321F0E7
:1038900088E00E944B0B11CD88E00E94AD0B0DCD4E
:1038A000CF911F910F91FF90EF900895AA1BBB1B22
:1038B00051E107C0AA1FBB1FA617B70710F0A61B30
:1038C000B70B881F991F5A95A9F780959095BC0151
:1038D000CD010895A1E21A2EAA1BBB1BFD010DC04C
:1038E000AA1FBB1FEE1FFF1FA217B307E407F507B0
:1038F00020F0A21BB30BE40BF50B661F771F881F8C
:10390000991F1A9469F760957095809590959B0121
:08391000AC01BD01CF010895D7
:1039180064207F526563656976656420556E6B6EB9
:103928006F776E204D4944493A203078000A0D00DF
:1039380004050607111210130409050A06070B11DE
:103948000C120D1013201B191C1A180F0C0E0B0D3E
:103958000A0920191A180C0B0A09222125232019F3
:103968001A18241B1C0F0E0D04030A0C0B0908015E
:10397800020026271D1E1F101211131415161705F5
:10398800060700070E091C1B1215383F3631242381
:103998002A2D70777E796C6B6265484F4641545387
:1039A8005A5DE0E7EEE9FCFBF2F5D8DFD6D1C4C3F7
:1039B800CACD90979E998C8B8285A8AFA6A1B4B3E7
:1039C800BABDC7C0C9CEDBDCD5D2FFF8F1F6E3E457
:1039D800EDEAB7B0B9BEABACA5A28F888186939447
:1039E8009D9A2720292E3B3C35321F1811160304B7
:1039F8000D0A5750595E4B4C45426F6861667374A7
:103A08007D7A898E878095929B9CB1B6BFB8ADAA06
:103A1800A3A4F9FEF7F0E5E2EBECC1C6CFC8DDDA06
:103A2800D3D4696E676075727B7C51565F584D4A76
:103A38004344191E171005020B0C21262F283D3A66
:103A480033344E49404752555C5B7671787F6A6DD6
:103A580064633E39303722252C2B0601080F1A1DC6
:103A68001413AEA9A0A7B2B5BCBB9691989F8A8D36
:103A78008483DED9D0D7C2C5CCCBE6E1E8EFFAFD26
:103A8800F4F3010409050A06070B110C120D1013B3
:00000001FF
